S2140F00007A0C1AB600000000000000000000000086
S20C0F00100000000000000000D4
S2140C138801340003026E20003814FFC42001381400
S2140C1398FFC03E1C000200000300281000000300DB
S2140C13A8146430020730FFFC1825000101340016BF
S2140C13B800FF0000000040000060000080000200F3
S2140C13C8000400000600000000000020000040009A
S2140C13D800600000800000A00000C00000E00001D3
S2140C13E800000200000300000400000500000600D0
S2140C13F800070000000000004000006000008000AD
S2140C1408020000040000060000080000084000085F
S2140C141860000880000A00000C00000E00000000A7
S2140C1428000040000060000080000200000400007D
S2140C14380600000800000A00000C00000E00000E53
S2140C144800003711B6F83706B6FE27F73701B0EEA8
S2140C1458F50F27FAF500379CF50C379E37BE0000BB
S2140C146837BC000027F7F500379C37BC000027F57B
S2140C147837FA0006F50C379E37BE0000277527F797
S2140C1488F80CBC121775FA4176FC177AFA411775E0
S2140C1498FA1376FB177AFA13B012F60B1775FA418D
S2140C14A87703177AFA411775FA137704177AFA132B
S2140C14B8379C27F73902FA13274C37B5FFFF8A00F3
S2140C14C88A0027F7000000003902FA13274C37E584
S2140C14D814CE8A0037B5000327F9FF6437E514CC19
S2140C14E83802FA13274C8400B6023C0237ACB00418
S2140C14F837B5FFFB37FA000627F7000037BE0000A3
S2140C150837BC00003902FA13274C37E515028A0057
S2140C15183802FA13274C850227F737B5808037EA46
S2140C15281502FA0C150437B8BDBD3787008837B8CE
S2140C15382A2A3787008037B5909037EA1502FA0CB6
S2140C1548150437B8889D3787006C37350000390284
S2140C1558FA13274C37B5AAAA37CA555537B5555571
S2140C156837CA2AAA37B5909037CA55553802FA138F
S2140C1578274C850237B84471B72437B84470B71E61
S2140C158837B88895B71837380001B60237F500080B
S2140C1598B0222735000837B5FFFE37FA00067A0C56
S2140C15A81ABE7C0137380001B60637FA0008F5086B
S2140C15B8379CB09637B5000137FA000827F537FA86
S2140C15C800067A0C1ABE3711B6F83706B6FE27F799
S2140C15D83701B0EE27757CFFB712CB0202F6550022
S2140C15E84A0655014A073D023EFFB6E47501B0FEB1
S2140C15F8370527F7273500067500177AFA4137B5E9
S2140C1608008036BE75FF177AFA4137B5010137FAEE
S2140C1618F92437B5FF0036AAF50D379C37BC000001
S2140C162845017816B6008B02020A37350001377A60
S2140C1638000637800050F50C379D37BD1388377574
S2140C16480014375A000437BE0019FA0C15DC370696
S2140C1658B7201709080037B50300FA0C15CE2775FE
S2140C16687CFFB718CB0102F64506C50737FA0012F9
S2140C167827350006B00E37350002377A0006B00458
S2140C168837350003377A00067A0C1ABE37F5000889
S2140C169837B8BDBD3787003A37B82A2A378700C807
S2140C16A837B844713787012C37B888953787013295
S2140C16B837B844703787018437B80001378701304C
S2140C16C837B8889D3787014437B5FFF937FA0006CF
S2140C16D87A0C1ABEFA0C146E3735001937B540401A
S2140C16E88A0027F58A0037B5000727F9FD5237B563
S2140C16F8000037EA14CC37B5C0C037EA14CEFA0C5B
S2140C170814D027360006BD0637350019F808B70A70
S2140C1718B0C67CFFB74C27F537FA0006B0BAFA0CF9
S2140C1728146E373503E837B520208A008A0037B59B
S2140C1738271027F9FD0A37B5FFFF37EA14CC37B55B
S2140C1748A0A037EA14CEFA0C14D027360006B60634
S2140C1758373503E8F808B70AB0E07CFFB70427F576
S2140C176837FA0006B0BC7A0C1ABEFA0C146E37356B
S2140C177807D0FA0C14BC37B530308A008A00380209
S2140C1788FA13274C37B5271027F9FCB437B5FFFFE3
S2140C17988400B7087CFFB6E837B5FFFD37FA0006B5
S2140C17A87A0C1ABE3902FA13274C37B550508A00F1
S2140C17B837B520208A0037B5D0D08A003802FA13FD
S2140C17C8274C8500F980B7F6F920B70437B5FFFD26
S2140C17D837FA000627F7FA0C146E37BE13BA3735E5
S2140C17E80007B032FA0C146E37BE13CF3735000F1D
S2140C17F8B024FA0C146EFA0C14BCF508FA0C1488FF
S2140C1808FA0C14BC37BE13FC3735000DB008FA0CAE
S2140C1818146E37BE14263735000B7CFFE500379C54
S2140C18283E01EC00FA0C1488FA0C17AC27360006A6
S2140C1838B6043E0237380000BEDC7A0C1ABE7A0CA8
S2140C18481ABE37F5000837B8BDBD3787004437B819
S2140C18582A2A3787003C37B84471378700B637B81A
S2140C18688895378700AE37B84470378700A637B8E0
S2140C187800013787009E37B8889D3787009637B59E
S2140C1888FFF937FA00067A0C1ABEF50C379D37BDE9
S2140C1898000027F7FA0C1892FA0C146EFA0C14BC03
S2140C18A83735001917FE00103EFF3902FA13274C7D
S2140C18B817F5000E17FC000C379C37B540408A000D
S2140C18C895008A0037B5000727F9FB74950017BEF4
S2140C18D8001037BE000037EA14CC37B5C0C037EA5C
S2140C18E814CEFA0C14D027360006B61637AC17FAF0
S2140C18F8000E17BC000C3735001917FE00103EFFFB
S2140C1908B70C3D02B0A07CFFB70427F537FA0006E3
S2140C1918B0947A0C1ABEFA0C1892FA0C146E17FEBF
S2140C19280010373500033902FA13274CFA0C14BC8E
S2140C1938F508379CFA0C14BC3EFFB77E3902FA132E
S2140C1948274C17F5000E17FC000C17FA000FFA0CAC
S2140C1958148837B550508A0037B540408A00950031
S2140C19688A003802FA13274C8500F980B7F68500EA
S2140C1978F910B7247CFFB6C037B5FFFC37FA00065B
S2140C19887A0C19C637B5FFFF8A0085009800B70889
S2140C199837B5FFFC37FA00067A0C19C6373500033C
S2140C19A817F5000F379C27F537FA00063D023C0260
S2140C19B817BC000C37AC17FA000E7A0C19407A0CC8
S2140C19C81ABEF50E379C75AA37BC55554A00755580
S2140C19D837BC2AAA4A0075A037BC55554A007A0C5B
S2140C19E81ABEF50E379C75AA37BC55554A00755560
S2140C19F837BC2AAA4A00758037BC55554A0075AAC2
S2140C1A0837BC55554A00755537BC2AAA4A00752066
S2140C1A1837BC55554A007A0C1ABE37B509C427F98F
S2140C1A28FA1E27F7FA0C189217FE001017F5000E78
S2140C1A3817FC000C379C17BC000627380006003F1E
S2140C1A4855004A003D013EFFB71817BC00163775FF
S2140C1A580016377000063738003FBD02360C3C01BE
S2140C1A68B0D03C01B0D6FA0C1A767A0C1A843735F4
S2140C1A7802587CFFB6F84800B6F827F7FA0C189206
S2140C1A882735000617FE001017F5000E17FC000C7D
S2140C1A98379C55004800B6063D013C013EFFB7068C
S2140C1AA8B0EC37B5FFFA37FA00067A0C1ABEF50F03
S2140C1AB8379F37BF03FC37A6FA0C145837F5000ABD
S2140C1AC837B800013787FA5037B800023787FBBAA1
S2140C1AD837B800033787FD6837B800043787FB121A
S2140C1AE837B800053787FF3A37B800063787FEF051
S2140C1AF837B800073787FEC837B5FFF937FA000638
S2060C1B08B0B06A
S804000000FB
